:100000000C942E050C9449050C9491160C94B5167D
:100010000C9449050C94F2110C9449050C94490573
:100020000C9449050C9449050C94FC090C94490561
:100030000C9449050C9449050C9449050C94490508
:100040000C9449050C9449050C9449050C944905F8
:100050000C9449050C9449050C94B8134156522050
:10006000427574746572666C792047434300546925
:100070006D6500436C6F636B0041646A7573742037
:10008000436C6F636B004368616E676520436C6F00
:10009000636B20466F726D6174004461746500414A
:1000A000646A7573742044617465004368616E67A7
:1000B00065204461746520466F726D6174004D75F2
:1000C000736963004E616D6500456E746572206EE4
:1000D000616D650054656D7065726174757265005F
:1000E000566F6C74616765004C69676874004F7087
:1000F00074696F6E7300446973706C617900416458
:100100006A75737420636F6E7472617374004272E7
:100110006F777365207365676D656E747300446FE8
:10012000776E6C6F6164204E616D6500426F6F7415
:100130006C6F6164657200506F77657220536176F1
:1001400065204D6F6465004175746F20506F776551
:10015000722053617665000A045A0A020B0A0514DC
:100160000B030A14040A14021514030A14052815B3
:10017000041B15021615031415051B170419170186
:10018000181703161705191904171901241903164E
:100190001905171B04151B021C1B03141B05151D39
:1001A000041F1D011E1D031C1D051F1F041D1F0113
:1001B000201F031C1F051D28041428022A28030AD7
:1001C00028053229022A2903283204283202333230
:1001D000030A32053C35043735013635033335051E
:1001E000373704353701383703333705353C0432A8
:1001F0003C023D3C030A3C054646043C4602474659
:10020000030A46055050044650025150030A500557
:100210005A5A04505A025B5A030A5A050A5B04628E
:100220005B025C5B035A5B055E5C015D5C035B5ECD
:10023000045B5E025F5E035A5E056060045E6002FE
:100240006160035A60056262046062026362035A7D
:1002500062055B0000000A5C0000000B000029073B
:10026000146E0000001573000000160000080E1741
:10027000790000001800007C0E19860000002400A0
:1002800000900F1B9A0000001C0000D60F1D9F005D
:1002900000001E000085101FAB000000200000AE13
:1002A0001128BE0000002A0000FC0B2B0000840C6B
:1002B00032C4000000330000BF0735C9000000371A
:1002C0001E010000360000110838000011093CD45E
:1002D0000000003D0000441946E000000047000017
:1002E0007B1950E80000005100009E195AEE0000F2
:1002F000005BF60000005CFE0000005D00000413DF
:100300005E2C0100005F00006306603701000061A1
:10031000000081066247010000630000A2060000A1
:100320000000004A756D7020746F20626F6F746CEE
:100330006F6164657200507265737320656E7465D9
:100340007220746F20736C656570004F6666004F95
:1003500066660077616974696E6720666F722069EE
:100360006E707574206F6E205253323332005465B4
:100370007374004C65667400557000526967687448
:1003800000446F776E00536F756E64004C434420D9
:1003900074657374004572726F722054656D706578
:1003A000726174757265004572726F7220566F6C5F
:1003B00074616765004C69676874004572726F729A
:1003C0002044617461666C617368004675722045F3
:1003D0006C69736500030008007B01080092010846
:1003E000007B010800920108007B010800FA010867
:1003F00000AA010800DE010400380208000100081C
:1004000000BC030800F602080038020400FA0108E4
:100410000001000800F60208005A020800FA010470
:1004200000DE01080001000800F60208007B010858
:1004300000920108007B010800920108007B01087E
:1004400000FA010800AA010800DE010400380208D1
:100450000001000800BC030800F60208003802048E
:1004600000FA01080001000800F6020800DE010899
:1004700000FA0104003802000001005475726B6537
:1004800079206D617263680003001000A4021000FF
:10049000F602100024031000F60204007E02100091
:1004A000380210007E021000A40210007E02040038
:1004B000FA011000DE011000FA011000180210000D
:1004C000FA011000520110007B011000920110008F
:1004D0007B011000520110007B01100092011000FE
:1004E0007B0104003F0108007B0108003F01200060
:1004F000AA0120007B011000520108007B010800C6
:10050000AA0108007B012000AA0120007B01100045
:10051000520108007B010800AA0108007B012000AD
:10052000AA0120007B011000520108007B01080095
:10053000AA010800C3010400FA0100000100536988
:1005400072656E65310000002000900120008D0171
:1005500020008A0120008701200084012000810101
:1005600020007E0120007B01200078012000750121
:100570002000720120006F0120006C012000690141
:1005800020006601200063012000600120005D0161
:1005900020005A0120005701200054012000510181
:1005A00020004E0120004B012000480120004501A1
:1005B0002000420120003F0120003C0120003901C1
:1005C00020003601200033012000300120002D01E1
:1005D00020002A0120002A0120002D0120003001E6
:1005E00020003301200036012000390120003C01A9
:1005F00020003F0120004201200045012000480169
:1006000020004B0120004E01200051012000540128
:100610002000570120005A0120005D0120006001E8
:1006200020006301200066012000690120006C01A8
:1006300020006F0120007201200075012000780168
:1006400020007B0120007E01200081012000840128
:100650002000870120008A0120008D0120009001E8
:1006600000000100536972656E65320003000400EA
:10067000DE0104003F010000010057686973746CDB
:10068000650000002000C8002000C3002000BE005C
:100690002000B9002000B4002000AF002000AA0014
:1006A0002000A5002000A00020009B002000960054
:1006B0002000910020008C00200087002000820094
:1006C00020007D00200078002000730020006E00D4
:1006D0002000690020006400080001002000C8001C
:1006E0002000C3002000BE002000B9002000B4009C
:1006F0002000AF002000AA002000A5002000A000DC
:1007000020009B00200096002000910020008C001B
:10071000200087002000820020007D0020007D0056
:10072000200082002000870020008C002000910023
:100730002000960020009B002000A0002000A500C3
:100740002000AA002000AF002000B4002000B90063
:100750002000BE002000C3002000C80000000000F0
:10076000504C4159494E470044444D4D5959004D54
:100770004D444459590059594D4D44440004050213
:100780000300010405000102030001020304053215
:1007900034480031324800313248003234480032A7
:1007A00034480031324800510A802A0000000A51C2
:1007B0000A000059551801111E111B500B411B4115
:1007C0001F1101511F511B0000000000000000001C
:1007D0000000000000510F913941149131411E4138
:1007E0000E411D500F80201015488640147805706A
:1007F000855115510E5195518E21908120501548EB
:100800004450C528C0282009500000000000000006
:1008100000000009090909090A0A0B080108010872
:10082000010801080110021002200426031C031213
:10083000030703FD02F202E702DC02D002C502B99F
:1008400002AD02A102950289027C02700263025786
:10085000024A023E023202250219020C020002F490
:1008600001E801DC01D001C401B801AD01A201968B
:10087000018C01810176016C01620158014E014435
:10088000013B0132012901200117010F010701FF7E
:1008900000F700F000E900E100DB00D400CD00C764
:1008A00000C100BB002F03390342034B0353035C19
:1008B0000364036C0373037B03820388038F039534
:1008C000039B03AA03A703A403A1039E039B03980E
:1008D00003940391038D038A03860382037E037BC3
:1008E00003770372036E036A03660361035D0358B3
:1008F0000353034F034A03450340033B03360330CE
:10090000032B03260320031B0315030F030A030411
:1009100003FE02F802F202EC02E602DF02D902D381
:1009200002CC02C602BF02B902B202AC02A5029E0C
:1009300002970291028A0283027C0275026E0268AB
:100940000261025A0253024C0245023E0237023053
:1009500002290222021B0215020E0207020002F9FE
:1009600001F201EC01E501DE01D801D101CB01C4A6
:1009700001BE01B701B101AA01A4019E0198019233
:10098000018C01860180017A0174016E01680163A6
:10099000015D01580152014D01470142013D0138FD
:1009A0000133012E01290124011F011A0115011132
:1009B000010C0108010301FF00FB00F600F200EE4C
:1009C00000EA00E600E200DE00DB00D700D300CF43
:1009D00000CC00C800C500C200BE00BB00350060EE
:1009E000008000B0001D013D015A017A019701B954
:1009F00001DA01F901160240026D028202A202EF41
:100A0000023203B003F2031D5A3440E17A34406AE3
:100A1000BC344091ED34407D3F3540A47035402DCD
:100A2000B23540F2D23540B6F335403F35364066F8
:100A30006636408D97364017D93640643B3740EED6
:100A40007C374014AE37409EEF3740B0723840E9F3
:100A500026394021B03A4093183C400011241FBE73
:100A6000CFEFD4E0DEBFCDBF11E0A0E0B1E0EEE912
:100A7000F5E302C005900D92A636B107D9F712E052
:100A8000A6E6B1E001C01D92A630B107E1F70C94D3
:100A90004B050C940000CFEFD4E0DEBFCDBFCC24DB
:100AA0008AE0D82ED092A4010CE510E0EE24FF24B9
:100AB0000E943F067894C0916701CC2309F048C09A
:100AC0000115110549F061E0C8010E9482128C2FC6
:100AD0000E94F31200E010E00E940D17682FE1144D
:100AE000F10471F0F701099511C0F901E95AFD4FC0
:100AF00005911491F901E75AFD4FE590F49028C053
:100B0000882329F08091A4010E941506D82E809197
:100B1000A401D816E9F0D092A40140E065E0E6E532
:100B2000F2E084918823A1F0469F90011124F901FD
:100B3000EA5AFD4F94918091A4019817B1F24F5F4A
:100B4000469FF0011124EA5AFD4F8491882361F7F2
:100B500080910101882371F09091910180910001B1
:100B6000981740F08AE08093A4011092910181E0EF
:100B7000809367011F9904C01E9902C00E949F0ABA
:100B800093B19095907D8CB180958C70982B9C152D
:100B900021F0C92E109266010BC0992349F0809173
:100BA0006601813011F40E94D91683E080936601BA
:100BB00080916801882369F580916901882349F54E
:100BC00090916701992329F08091E4008F778093B9
:100BD000E40083B7817F866083BF85B7816085BF6E
:100BE000889585B78E7F85BF9923E9F01E991BC034
:100BF0001092670140E0ECEEF0E011924F5F44315B
:100C0000E0F38091E40080688093E4000E940D1777
:100C10000AC083B7817F83BF85B7816085BF889510
:100C200085B78E7F85BF13BE46CF582F982F40E0E3
:100C300023E0E7E5F1E084918823F1F0429F900101
:100C40001124F901E95AFE4F8491851759F4F901ED
:100C5000E85AFE4F8491861729F4F901E75AFE4FAE
:100C600094910AC04F5F23E0429FF0011124E95A9A
:100C7000FE4F8491882311F7892F992708950E94A8
:100C80005C0790E89093610083E08093610090BFDF
:100C900087E080937F008FE085B980EF8EB9259A39
:100CA0002D9A0E9479160E94C90D0E94E4098CE0D9
:100CB00090E00E94C3090E94EC140E94FE14289A3E
:100CC0000E9463130895982F80910201882341F0B8
:100CD0001092020161E083E293E00E9482120EC052
:100CE000913021F488E180936000FFCF933031F49C
:100CF00081E0809302018EE590E008958FE590E019
:100D00000895982F80910301882341F010920301E8
:100D100061E086E393E00E94821211C0913039F4C1
:100D200090936701909303018AE090E008959330D7
:100D300031F481E08093030180E690E0089581E63C
:100D400090E00895EF92FF920F931F93CF93F0904E
:100D50000401FF2069F010920401809101018823B1
:100D600019F08091000134C061E08BE493E029C068
:100D7000813029F48093040182E690E054C08430ED
:100D800059F4809100018B5F809300018B35E0F076
:100D90008AE58093000145C0853009F042C080910A
:100DA0000001882319F08550809300018091000193
:100DB000853050F4F0920101F092000161E08FE47F
:100DC00093E00E9482122DC091E0E92EE092010191
:100DD0000E941917C82F082F0F70005DC295CF70A1
:100DE000C05D6DE480E00E94E11269E481E00E9450
:100DF000E1126EE482E00E94E11260E283E00E9470
:100E0000E1126C2F84E00E94E112602F85E00E94C5
:100E1000E11260E086E00E94E11260E081E00E9461
:100E2000F61283E690E0CF911F910F91FF90EF9023
:100E3000089501972FEF8F3F920751F020E00000B7
:100E40002F5F2D37E0F301972FEF8F3F9207B1F718
:100E50000895982F80910501882319F110920501BA
:100E600062E580E00E94E11265E481E00E94E11207
:100E700066E582E00E94E11260E283E00E94E112F6
:100E800060E384E00E94E11266E385E00E94E112E3
:100E900060E086E00E94E11260E081E00E94F612CC
:100EA00008C0933031F481E0809305018AE090E03E
:100EB00008958BE090E00895CF93C0E080E88093A0
:100EC000610083E080936100C093700088E08093AC
:100ED000B60088EC8093B300C0936E0081E08093ED
:100EE00081008093B0008091B600282F33272170B5
:100EF00030708091B600992784709070282B392B20
:100F0000232B89F788EE93E00E941907F8948FEF5E
:100F100086BB87BB10928500109284001092B200AD
:100F200087B38823E9F310928100789486B38823ED
:100F300019F02FEF3FEF0AC0909184008091850057
:100F4000282F3327322F2227290F311D88E12B36F6
:100F5000380724F080916600815006C0285E374132
:100F600034F4809166008F5F8093660001C0C1E019
:100F700081E080938100CC2349F2CF910895CF93F3
:100F8000DF93CDB7DEB722970FB6F894DEBF0FBE62
:100F9000CDBF282F80E091E089839A83809106015C
:100FA000882321F110920601F999FECF89819A8157
:100FB00092BD81BDF89A80B5682F772760936A014A
:100FC000862F8150893130F010926A0181E480933C
:100FD000A5010EC041E051E085EA91E00E94BF14F6
:100FE00061E085EA91E00E94B51210C0223031F430
:100FF00081E08093060185E390E00AC0233031F45C
:1010000081E08093060182E390E002C083E390E0F8
:1010100022960FB6F894DEBF0FBECDBFDF91CF9101
:1010200008951F93CF93DF93CDB7DEB722970FB606
:10103000F894DEBF0FBECDBF182F80E091E089830A
:101040009A8380910701882391F041E051E06091FB
:101050006A0185EA91E00E94BF1480916A018823A9
:1010600019F0815080936A011092070155C0909148
:101070006A0190936B0185E080937201382F492FAC
:10108000E92FFF27EB55FE4F2081822F80528B35B1
:1010900040F49F3F31F0E32FFF27E459FE4F2083B8
:1010A00006C0E32FFF27E459FE4F80E280833150D2
:1010B000942F91503F3F19F73093720190936B0139
:1010C00060916C0180E00E94E11260916D0181E00D
:1010D0000E94E11260916E0182E00E94E112609133
:1010E0006F0183E00E94E1126091700184E00E9430
:1010F000E112809171018068682F85E00E94E11201
:1011000060E086E00E94E112112311F00E940113B9
:1011100060E081E00E94F612112311F00E94011399
:101120001430D1F480916A01E82FFF27EB55FE4F70
:101130009081292F21502083892F82528F3030F1C6
:101140009B53973010F489E33BC02B3518F42032C1
:1011500008F05BC08AE534C01530D1F480916A0193
:10116000E82FFF27EB55FE4F9081292F2F5F20831B
:10117000892F80528F3010F480E322C0995397302A
:10118000F0F02B3518F4203208F03FC080E218C090
:10119000133041F480916A018823B9F18150809322
:1011A0006A0133C0123071F480916A01893168F5A7
:1011B0008F5F80936A01E82FFF27EB55FE4F81E494
:1011C000808323C0113009F520916A012F5F20939D
:1011D0006A01E22FFF27EB55FE4F1082F999FECFEF
:1011E00089819A8192BD81BD20BDFA9AF99A41E028
:1011F00051E060916A0185EA91E00E94911481E0DA
:101200008093070183E390E002C086E390E022969A
:101210000FB6F894DEBF0FBECDBFDF91CF911F9107
:1012200008951F93CF93DF93CDB7DEB722970FB604
:10123000F894DEBF0FBECDBF182F80E091E0898308
:101240009A83809108018823B1F0F89480E8809314
:10125000610082E080936100789460E083E593E030
:101260000E9482121092080110928C018091C60097
:1012700081E0809369018091C00087FF66C0809102
:10128000C60090918C018D3061F0993108F05DC0FD
:10129000E92FFF27ED58FE4F80839F5F90938C01CD
:1012A00054C0F89480E88093610083E080936100EB
:1012B0007894992309F445C0E92FFF27ED58FE4F94
:1012C000108210928C01809173018823A1F090818B
:1012D000E92FFF27DF01AD58BE4F8C91EB55FE4F34
:1012E00080839F5FE92FFF27ED58FE4F8081882381
:1012F00079F790938C0180918C01E82FFF27EB55B3
:10130000FE4F108281E08093080120916A01F999D3
:10131000FECF89819A8192BD81BD20BDFA9AF99A4A
:1013200041E051E060918C0185EA91E00E949114C6
:1013300080918C0180936A011092690183E390E0AF
:1013400018C081E0809308010FC0112381F081E073
:1013500080930801F89480E88093610083E0809393
:10136000610078941092690187E390E002C088E3FD
:1013700090E022960FB6F894DEBF0FBECDBFDF918E
:10138000CF911F9108959C01832F99278093C500C9
:101390002093C40082E08093C00080E18093C1006C
:1013A00086E08093C2000895982F8091C00085FF49
:1013B000FCCF9093C60008958091C00087FFFCCFBA
:1013C0008091C6009927089590E0E2ECF1E0119237
:1013D00011929F5F9430D8F390E0EEEBF1E08FEF45
:1013E00081939F5F9430D8F382E080936E0086E211
:1013F00087BD8CE084BD08951F920F920FB60F92A7
:1014000011240F931F932F933F934F935F936F93E9
:101410007F938F939F93AF93BF93CF93EF93FF935C
:10142000C0E002EC11E0D801ED91FD918D01309703
:1014300009F00995CF5FC430B0F3C0E0EEEBF1E006
:1014400080818F3F21F0882311F081508083CF5F0E
:101450003196C430A8F3FF91EF91CF91BF91AF9136
:101460009F918F917F916F915F914F913F912F91BC
:101470001F910F910F900FBE0F901F901895AC0108
:1014800020E0E2ECF1E0819191918417950761F001
:101490002F5F2430C0F320E0E2ECF1E08081918105
:1014A000892B29F44083518381E090E008952F5FD8
:1014B0003296243098F380E090E008959C0140E05B
:1014C000E2ECF1E0808191818217930729F4108288
:1014D000118281E090E008954F5F3296443090F39E
:1014E00080E090E0089590E0E92FFF27E254FE4F5E
:1014F00080819F5F8F3F21F41082892F9927089563
:10150000943090F380E090E00895F894E82FFF275E
:10151000E354FE4F608378940895F894E82FFF27F2
:10152000E354FE4F8081789499270895F894E82F2A
:10153000FF27E354FE4F8FEF8083789408951F9325
:10154000CF93DF93C0E0C09370006C2F8EE693E0E2
:101550000E9482120E940D178130E1F760E083E75C
:1015600093E00E9482120E940D178330E1F760E041
:1015700088E793E00E9482120E940D178430E1F701
:1015800060E08BE793E00E9482120E940D17823088
:10159000E1F760E081E893E00E9482120E940D175B
:1015A0008530E1F760E086E893E00E9482120E94B5
:1015B0000D178130E1F780E88093800081E180930E
:1015C0008100809181008160809381001092890068
:1015D00080E580938800C8ECD0E08D2F992787FDA7
:1015E0009A9580938700C09386008EE190E00E94D8
:1015F00019072597C436D10584F710928000109200
:10160000810060E08CE893E00E9482121C9BFECF78
:101610000E940D178130E1F78091E400877F80936D
:10162000E40090E0ECEEF0E08FEF81939F5F943167
:10163000D8F31C9BFECF84E690E00E9419071C990A
:10164000FECF8091E40088608093E40080E00E94F7
:101650004A170E945217EC01C45CD140C738D1052B
:10166000B0F060E085E993E00E9482120E94BC0B1A
:101670000E940D17C82F8130D9F70E948A1760E0A9
:101680008C2F0E94F6120E940D178130E1F781E045
:101690000E944A170E945217EC01CA52D140679724
:1016A000B0F060E087EA93E00E9482120E94BC0BD7
:1016B0000E940D17C82F8130D9F70E948A1760E069
:1016C0008C2F0E94F6120E940D178130E1F760E026
:1016D00085EB93E00E9482120E940D178130E1F7A2
:1016E00082E00E944A170E9452170E948A17000047
:1016F00060E081E00E94F6120E940D17813099F798
:10170000289A289810E0C0E0D0E0412FBE0181E087
:101710000E94C0151F5F21961233B8F361E070E09C
:1017200081E00E940C16289A289860E070E081E021
:1017300090E00E943D1610E080E00E94F714181718
:1017400061F060E08BEB93E00E9482120E94BC0B80
:101750000E940D178130E1F703C01F5F123360F361
:10176000289A81E00E9429070E940D178130E1F735
:1017700088E180936000FFCF1F9380E88093800012
:1017800081E180938100809181008160809381005C
:101790001092890080E58093880011E01093870003
:1017A0008FE38093860082E390E00E9419071093F4
:1017B00087008EED809386008CE291E00E941907ED
:1017C00010928000109281001F91089580E880930C
:1017D000800080E18093810080918100816080930E
:1017E000810010928900809121018093880086E019
:1017F0009DE00E943F0A0895CF93C82F8091220157
:101800008823E9F01092220180918F01E82FFF27B1
:10181000EE0FFF1FEB5EFE4F61E0808191810E9421
:10182000821280918F01E82FFF27EE0FFF1FE75FE5
:10183000FE4F808191819093CB018093CA01C43087
:1018400009F580918F018823C9F4E1E0E0938F01CD
:101850008091170190911801892B71F02E2F2F5F25
:10186000E22FFF27EE0FFF1FEB5EFE4F808191817D
:10187000892BA9F720938F0180918F01815080934C
:101880008F0113C0C53069F580918F018F5F809300
:101890008F01E82FFF27EE0FFF1FEB5EFE4F8081C9
:1018A0009181892B11F410928F0180918F01E82F83
:1018B000FF27EE0FFF1FEB5EFE4F61E080819181FD
:1018C0000E94821280918F01E82FFF27EE0FFF1FE9
:1018D000E75FFE4F808191819093CB018093CA0195
:1018E0000FC0C13029F4C09322018BE290E00AC0FE
:1018F000C33031F481E08093220188E290E002C09D
:101900008AE290E0CF9108951F93CF93182F809192
:101910002301882379F01092230110928E010E94F6
:10192000E60B61E080E697E00E94821281E08093FE
:1019300068010DC0C0916801CC2349F486E09DE0A8
:101940000E945E0AC0938000C093810054C014308E
:1019500041F480912101803510F080E50BC08B5F50
:1019600009C0153079F4809121018B3010F486E0A4
:1019700001C085508093210110928900809121013E
:1019800080938800113029F580916801882399F0AF
:1019900010926801809181008E7F8093810086E0A3
:1019A0009DE00E945E0A10928000109281002D9AA4
:1019B0001093230123C080938D0110938E010E9408
:1019C000E60B612F80E697E00E9482121093680177
:1019D00018C01330B1F410926801809181008E7F9D
:1019E0008093810086E09DE00E945E0A1092800054
:1019F000109281002D9A81E0809323018AE290E089
:101A000002C08BE290E0CF911F9108950F931F9336
:101A1000CF93DF9380918E01882381F480938D0191
:101A2000E091CA01F091CB010190F081E02D859108
:101A300094918093900181E080938E018091900138
:101A4000882309F09EC080918D01882321F0815068
:101A500080938D018CC020918E01E22FFF27EE0F25
:101A6000FF1F0091CA011091CB01E00FF11F0190FF
:101A7000F081E02DAF0185919491C22FCF5F892B2A
:101A800009F450C0FA012591349180E290E0B90147
:101A90000E94BB1A60938D01C0938E0140E050E01C
:101AA000EC2FFF27EE0FFF1FE00FF11F0190F081D9
:101AB000E02D259134912130310509F4A90180E010
:101AC00090E02130310509F4C901482B592B452BF1
:101AD00021F0809181008E7F03C080918100816020
:101AE00080938100F89480918E01E82FFF27EE0FFC
:101AF000FF1FE00FF11F80819181892F990F990BB2
:101B00001092850010928400809387000190F081EC
:101B1000E02D8591949180938600789480918E0138
:101B20008F5F10C0C0938E01EC2FFF27EE0FFF1FB9
:101B3000E00FF11F0190F081E02DC591D491CC23ED
:101B400021F081E080938E0112C0C0938E01C0937A
:101B50006801809181008E7F8093810086E09DE006
:101B60000E945E0AC0938000C09381002D9AE0918C
:101B7000CA01F091CB010190F081E02D8591949103
:101B800001C0815080939001DF91CF911F910F91FF
:101B9000089588EE93E00E941907F89480917000F0
:101BA0008E7F8093700088E08093B6001092B20020
:101BB0008091B00085608093B0008091B600282F9E
:101BC0003327217030708091B6009927847090700F
:101BD000282B392B232B89F78FEF87BB809170003F
:101BE00081608093700078941092CD011092D201A0
:101BF0008CE08093CC0189E08093CE018AE08093D1
:101C0000D10183E090E09093D0018093CF010895BB
:101C1000CF92DF92EF92FF920F931F93CF93C82E34
:101C200080914901882341F48091CC01E82FFF275E
:101C3000EF5CFE4F808102C08091CC010E94191799
:101C4000C82F2FE0D22ED82280E3D80EC295CF70B5
:101C5000C80F8091D2010E941917082F9FE0E92E2A
:101C6000E82280E3E80E02950F70080F8091CD0105
:101C70000E941917182F8FE0F82EF12280E3F80E3A
:101C800012951F70180F6C2F80E00E94E1126D2DCD
:101C900081E00E94E112602F82E00E94E1126E2D2D
:101CA00083E00E94E112612F84E00E94E1126F2D17
:101CB00085E00E94E11260E086E00E94E11281E08E
:101CC0000E94F31260E081E00E94F61283E0C816E1
:101CD00019F485E190E008C082E0C81619F487E1A4
:101CE00090E002C086E190E0CF911F910F91FF90AC
:101CF000EF90DF90CF900895CF92DF92EF92FF9216
:101D00000F931F93CF93C82E80915601882361F0C3
:101D10008091CC01809393018091D20180939401B2
:101D20008091CD018093950180914901882341F4F0
:101D300080919301E82FFF27EF5CFE4F808102C066
:101D4000809193010E941917C82F5FE0F52EF822A9
:101D500080E3F80EC295CF70C80F809194010E9465
:101D60001917182F4FE0E42EE82280E3E80E1295B1
:101D70001F70180F809195010E941917082F3FE0DE
:101D8000D32ED82280E3D80E02950F70080F6C2F47
:101D9000772780919601882309F4606880E00E948B
:101DA000E1126F2D772780919601882309F46068EE
:101DB00081E00E94E112612F7727809196018130A6
:101DC00009F4606882E00E94E1126E2D772780910D
:101DD0009601813009F4606883E00E94E112602F6F
:101DE000772780919601823009F4606884E00E9430
:101DF000E1126D2D772780919601823009F4606899
:101E000085E00E94E11260E086E00E94E11281E03C
:101E10000E94F312CC2011F00E94011360E081E0D7
:101E20000E94F61281E08093560184E0C81649F4BE
:101E300080919601E82FFF27ED56FE4F80818F5F3E
:101E40000BC085E0C81651F480919601E82FFF275A
:101E5000ED56FE4F8081815080832FC083E0C816ED
:101E600041F480919601882311F482E00DC08150E5
:101E70000BC082E0C81659F480919601823019F4A3
:101E8000109296011AC08F5F8093960116C081E070
:101E9000C81699F4F894809193018093CC018091B5
:101EA00094018093D201809195018093CD01789423
:101EB0001092960186E190E02BC0809193018F3FB4
:101EC00019F487E18093930180919301883110F098
:101ED00010929301809194018F3F19F48BE38093CA
:101EE0009401809194018C3310F0109294018091B0
:101EF00095018F3F19F48BE38093950180919501B3
:101F00008C3310F0109295011092560188E190E008
:101F1000CF911F910F91FF90EF90DF90CF90089598
:101F2000CF93C82F80915701882371F010925701E9
:101F300060914901613019F48FE897E003C061E0D6
:101F400083E997E00E948212C43081F460914901D4
:101F5000613029F41092490187E997E019C081E0C6
:101F600080934901682F8BE997E012C0C53099F43E
:101F700080914901882339F481E080934901682FD9
:101F80008FE997E005C01092490161E083EA97E08C
:101F90000E94821207C0C13029F4C093570186E124
:101FA00090E002C084E290E0CF910895CF92DF925A
:101FB000EF92FF920F931F93CF93C82F8091CF0181
:101FC0000E941917182FEFE0EE2EE82280E3E80EAA
:101FD00012951F70180F8091D1010E941917082FB8
:101FE0007FE0D72ED82280E3D80E02950F70080F1D
:101FF0008091CE010E941917F82E6FE0C62EC822DC
:1020000080E3C80EF694F694F694F694F80E809158
:102010009201E82FFF27EE0FFF1FE05BFE4F0190BC
:10202000F081E02D8491612F0E94E1128091920154
:10203000E82FFF27EE0FFF1FE05BFE4F0190F081BE
:10204000E02D319684916E2D0E94E11280919201D3
:10205000E82FFF27EE0FFF1FE05BFE4F0190F0819E
:10206000E02D32968491602F0E94E11280919201BE
:10207000E82FFF27EE0FFF1FE05BFE4F0190F0817E
:10208000E02D339684916D2D0E94E1128091920192
:10209000E82FFF27EE0FFF1FE05BFE4F0190F0815E
:1020A000E02D349684916F2D0E94E112809192016F
:1020B000E82FFF27EE0FFF1FE05BFE4F0190F0813E
:1020C000E02D359684916C2D0E94E11260E086E04F
:1020D0000E94E11281E00E94F31260E081E00E9420
:1020E000F612C33019F48BE190E007C0C23019F446
:1020F0008DE190E002C08CE190E0CF911F910F91B3
:10210000FF90EF90DF90CF900895FF920F931F9371
:10211000CF93F82E80915801882361F08091CF01F0
:10212000809397018091D101809398018091CE0195
:1021300080939901C0915901CC23C9F480919701F2
:102140000E941917182F082F0F70005D12951F702D
:10215000105D60E28C2F0E94E11260E281E00E943B
:10216000E11269E582E00E94E11269E535C0C13003
:10217000C9F4809198010E941917182F082F0F7029
:10218000005D12951F70105D60E280E00E94E11218
:1021900060E28C2F0E94E1126DE482E00E94E11265
:1021A0006DE41AC0C23019F5809199010E94191787
:1021B000182F082F0F70005D12951F70105D60E2E0
:1021C00080E00E94E11260E281E00E94E11264E49A
:1021D0008C2F0E94E11264E483E00E94E112612FDF
:1021E00084E00E94E112602F85E00E94E11260E02D
:1021F00086E00E94E11280E00E94F312FF2011F0BD
:102200000E94011360E081E00E94F61281E0809359
:10221000580184E0F81649F480915901E82FFF270E
:10222000E956FE4F80818F5F0BC085E0F81651F4B0
:1022300080915901E82FFF27E956FE4F8081815098
:10224000808332C083E0F81641F4809159018823DD
:1022500011F482E00DC081500BC082E0F81659F4F1
:1022600080915901823019F4109259011DC08F5F7D
:102270008093590119C081E0F816B1F4F894809167
:10228000970199279093D0018093CF018091980175
:102290008093D101809199018093CE01789410921E
:1022A00059018CE190E055C0809197018F3F19F45E
:1022B00083E68093970180919701843610F0109205
:1022C000970180919801882319F48CE080939801FC
:1022D000809198018D3018F081E080939801809171
:1022E000D1018230C9F42091CF013091D001C901D0
:1022F00083709070892B81F4C90164E670E00E94BC
:10230000BB1A892B39F4C90160E971E00E94BB1A3C
:10231000892B11F481E001C080E0882311F0EDE108
:1023200007C080919801E82FFF27EC5DFE4FE08108
:1023300080919901882311F4E0939901809199018A
:10234000E81718F481E080939901109258018EE10A
:1023500090E0CF911F910F91FF900895CF93C82FD8
:1023600080915A01882379F010925A01809192014C
:10237000E82FFF27EE0FFF1FE65BFE4F61E0808135
:1023800091810E948212C43049F48091920182307E
:1023900018F0109292010DC08F5F09C0C530B9F4DA
:1023A00080919201882311F482E001C081508093D2
:1023B000920180919201E82FFF27EE0FFF1FE65B4D
:1023C000FE4F61E0808191810E94821207C0C1307E
:1023D00029F4C0935A018CE190E002C080E290E0C1
:1023E000CF9108951F920F920FB60F9211242F9341
:1023F0003F934F935F936F937F938F939F93AF938D
:10240000BF93EF93FF938091CD018F5F8093CD01B8
:102410008C3309F066C01092CD019091D2019F5F7C
:102420009093D201809191018F5F809391019C33B1
:1024300008F457C01092D2018091CC018F5F809335
:10244000CC01883108F44DC01092CC018091CE01AE
:102450008F5F8093CE014091D1014230D9F4209119
:10246000CF013091D001C90183709070892B91F414
:10247000C90164E670E00E94BB1A892B39F4C901D6
:1024800060E971E00E94BB1A892B21F481E08093FE
:102490009A0102C010929A018091CE01282F332711
:1024A000E42FFF27EC5DFE4F908180919A01890F08
:1024B000912D911D82179307A4F491E09093CE0182
:1024C000842F890F8093D1018D3058F09093D101E2
:1024D0008091CF019091D00101969093D00180938B
:1024E000CF01FF91EF91BF91AF919F918F917F911C
:1024F0006F915F914F913F912F910F900FBE0F9071
:102500001F901895FC0180919B018823E1F7982F7B
:102510008491882391F0AF01A8EEB1E09F01F90109
:1025200084918D939F5F2F5F3F4F4F5F5F4FFA0105
:102530008491882311F0993190F3E92FFF27E85116
:10254000FE4F1082973048F081E08093D3011092C3
:10255000010283E080939C0104C01092D301109289
:10256000010281E080939B010895DC01E0919B01D1
:10257000EE23E1F79E2F8C91882359F0FD01A8EE00
:10258000B1E081918D939F5F8081882311F0993113
:10259000C0F3E92FFF27E851FE4F1082973048F033
:1025A00081E08093D3011092010283E080939C012B
:1025B00004C01092D3011092010281E080939B012C
:1025C0000895893128F4E82FFF27E851FE4F6083F2
:1025D0000895089590E0E8EEF1E080E281939F5F36
:1025E0009931D8F3089580939E01089590919B01AD
:1025F0009923E1F76093D3019093010280939B01AB
:10260000089510929D0108950F931F93CF93C82FA3
:1026100080915C01882321F00E94EA1210925C01F3
:1026200080915B010E941917182F082F0F70005D11
:1026300012951F70105D63E480E00E94E11264E572
:1026400081E00E94E11262E582E00E94E11260E214
:1026500083E00E94E112612F84E00E94E112602F6A
:1026600085E00E94E11260E081E00E94F612C43031
:1026700021F480915B018F5F05C0C53029F4809102
:102680005B01815080935B0180915B018F3F11F46E
:1026900010925B0180915B01803118F08FE0809394
:1026A0005B0180915B018F708093E700C13029F45A
:1026B000C0935C018CE590E002C08DE590E0CF9185
:1026C0001F910F91089580E00E94AE138FE08093D8
:1026D000E70087EB8093E50087E08093E60080ECDD
:1026E0008093E4008091E40088608093E40010927D
:1026F0009B010895E82F20E030E0663070F58A52A3
:10270000813558F4E13608F0EF7DEA52FF27EE0FED
:10271000FF1FE955F84F25913491A62FBB27A0FF45
:1027200002C05FE001C050EF6695E62FFF27EC5234
:10273000FE4F40E0922F9F7084E0369527958A9552
:10274000E1F7A0FF02C09295907F80818523892BBD
:10275000808335964F5F443068F3089581118FEF81
:1027600090E0E4EDF1E081939F5F9431E0F3089510
:102770001F920F920FB60F921124DF92EF92FF92E9
:102780000F931F932F933F934F935F936F937F9379
:102790008F939F93AF93BF93CF93EF93FF93DD24DA
:1027A0008091A101882361F480919F018F5F8093C4
:1027B0009F01843028F081E08093A101D0929F0195
:1027C00080916601833071F48091A0018F5F8093C6
:1027D000A001813148F081E0809366018FE0809311
:1027E000A00102C01092A00180915D0181508093F0
:1027F0005D019091D301992371F0882371F4809148
:102800009C01882321F481E080939B0106C08150C4
:1028100080939C0102C090930102FF2490919B0140
:10282000913009F056C080919D01853010F4EF2C55
:1028300001C0E92EC0E000E010E08091010299277C
:1028400087FD9095800F911F97FD17C0FF20A9F479
:1028500080910102E82FFF27E7FDF095E851FE4F38
:10286000E00FF11F8081DF2C87FF02C091E0D92E9D
:102870008F7721F4FC2EF39401C080E2DD2029F053
:10288000EE2019F06C2F80E201C06C2F0E947A13A9
:10289000CF5F0F5F1F4FC63080F2C0E0ACEEB0E0FC
:1028A000E4EDF1E081918D93CF5FC431D8F3809155
:1028B0009E01811181E08093F40081E0F81611F40B
:1028C0008AEF03C0809101028F5F80930102109212
:1028D0009B0180915D01882319F483E080935D0161
:1028E00080919D018A3019F410929D0103C08F5F81
:1028F00080939D01FF91EF91CF91BF91AF919F91F7
:102900008F917F916F915F914F913F912F911F9187
:102910000F91FF90EF90DF900F900FBE0F901F90E0
:102920001895CF93DF93CDB7DEB722970FB6F89403
:10293000DEBF0FBECDBFDC0149835A8320E02617DE
:10294000A8F4FD01E20FF11DE081F999FECF898124
:102950009A8192BD81BDE0BDFA9AF99A89819A81E6
:10296000019689839A832F5F261758F322960FB614
:10297000F894DEBF0FBECDBFDF91CF910895CF9306
:10298000DF93CDB7DEB722970FB6F894DEBF0FBE48
:10299000CDBFDC0149835A8320E02617A0F4FD0156
:1029A000E20FF11DF999FECF89819A8192BD81BD17
:1029B000F89A80B5808389819A81019689839A8368
:1029C0002F5F261760F322960FB6F894DEBF0FBE76
:1029D000CDBFDF91CF91089585B18F6085B984B166
:1029E000876084B981E08DBD8CE58CBD08958EBD76
:1029F0000DB407FEFDCF8EB599270895289A289823
:102A000087E50E94F71480E00E94F714482F5527AD
:102A1000CA018873907023E0959587952A95E1F710
:102A20009927FC01ED5EF74F249120930202FC01EF
:102A3000E80FF91FE55EF74F85919491909304029A
:102A400080930302CA010895CF93DF93EC01289A83
:102A50002898613009F583E50E94F714209102025D
:102A600080E190E0821B91099E0102C03695279576
:102A70008A95E2F7C9010E94F71480910202992712
:102A8000089702C0CC0FDD1F8A95E2F78C2F0E94B9
:102A9000F71480E00E94F714289A28980E94FE14E8
:102AA00087FFFCCFDF91CF910895CF93DF93EB01A8
:102AB00090E3289A28988130A1F484E50E94F714C5
:102AC00080E00E94F7148D2F99270E94F7148C2F15
:102AD0000E94F71480E00E94F71480E00E94F7142F
:102AE000982F892F9927DF91CF910895EF92FF9228
:102AF0000F931F93CF93DF93EB017A018901289AFB
:102B000028988130F9F484E50E94F71480E00E944F
:102B1000F7148D2F99270E94F7148C2F0E94F71419
:102B200080E00E94F714C0E0D0E0CE15DF0550F43D
:102B300080E00E94F714F80181938F012196CE1551
:102B4000DF05B0F3DF91CF911F910F91FF90EF90D0
:102B50000895CF93DF93EB01289A2898813069F488
:102B600084E80E94F71480E00E94F7148D2F9927C3
:102B70000E94F7148C2F0E94F714DF91CF910895D3
:102B80001F93CF93DF93EB01142F289A289881305D
:102B900081F484E80E94F71480E00E94F7148D2FDE
:102BA00099270E94F7148C2F0E94F714812F0E94FE
:102BB000F714DF91CF911F910895EF92FF920F9339
:102BC0001F93CF93DF93EB017A018901289A28980C
:102BD0008130D9F484E80E94F71480E00E94F71451
:102BE0008D2F99270E94F7148C2F0E94F714C0E0B4
:102BF000D0E0CE15DF0548F4F80181918F010E94E5
:102C0000F7142196CE15DF05B8F3DF91CF911F9110
:102C10000F91FF90EF900895CF93DF93EB01289AE7
:102C20002898813009F583E80E94F7142091020268
:102C300080E190E0821B91099E0102C036952795A4
:102C40008A95E2F7C9010E94F71480910202992740
:102C5000089702C0CC0FDD1F8A95E2F78C2F0E94E7
:102C6000F71480E00E94F714289A28980E94FE1416
:102C700087FFFCCFDF91CF910895EF92FF920F93E2
:102C80001F938C017B01289A289888E60E94F714EC
:102C90002091020280E190E0821B9109980102C01C
:102CA000369527958A95E2F7C9010E94F71480911D
:102CB00002029927089702C0000F111F8A95E2F7B8
:102CC0008F2D9927800F0E94F7148E2D0E94F714E4
:102CD00080E00E94F71480E00E94F71480E00E94D8
:102CE000F71480E00E94F7141F910F91FF90EF906E
:102CF000089527982698249885B1806D85B91DB8C8
:102D00008EB18C608EB98CE080936B0080ED8093E7
:102D10006C0080EC8CBB8DBB0E94730A8093050213
:102D200008951F920F920FB60F9211242F933F9385
:102D30004F935F936F937F938F939F93AF93BF93C3
:102D4000EF93FF930E94D916FF91EF91BF91AF913E
:102D50009F918F917F916F915F914F913F912F91B3
:102D60000F900FBE0F901F9018951F920F920FB6E5
:102D70000F9211242F933F934F935F936F937F9301
:102D80008F939F93AF93BF93EF93FF930E94D916B6
:102D9000FF91EF91BF91AF919F918F917F916F9133
:102DA0005F914F913F912F910F900FBE0F901F9009
:102DB000189523B12095207D8CB180958C70282B9F
:102DC000822F992786FF02C094E011C027FF02C01E
:102DD00095E00DC082FF02C093E009C083FF02C0EE
:102DE00092E005C084FF02C091E001C090E0992309
:102DF00079F08091A101882359F08091A301882363
:102E000029F49093A20181E08093A3011092A10183
:102E100080EC8CBB109291010895F8948091A301ED
:102E2000882321F08091A2011092A3017894992720
:102E30000895282F80E02A3020F08F5F2A502A3012
:102E4000E0F7992734E0880F991F3A95E1F7282B8E
:102E5000822F9927089520E030E0843628F02F5FF4
:102E60003F4F84568436D8F754E0220F331F5A95CB
:102E7000E1F78A3028F02F5F3F4F8A508A30D8F729
:102E800044E0220F331F4A95E1F79927282B392B6D
:102E9000C901089580937C0083E880937A000E94A2
:102EA0005217089540E050E08B9A839A80917A00FF
:102EB000806880937A0080917A00806480937A00A1
:102EC00080917A0084FFFCCF30E080917A008064AA
:102ED00080937A0080917A0084FFFCCF2091780063
:102EE000809179009927982F8827820F911D480F8C
:102EF000591F3F5F383048F383E0559547958A95D1
:102F0000E1F78B98839880917A008F7780937A008D
:102F1000CA0108959F92AF92BF92CF92DF92EF9233
:102F2000FF920F931F93CF93DF93C0E0D0E09924DB
:102F30000E9452179C0180917C00882309F099C05F
:102F400080916201833009F04CC083E02B32380756
:102F50008CF0AE01FA01EB55F74F859194918217F1
:102F6000930730F493944E5F5F4F99E1991590F772
:102F70006DE216C0E3E020323E078CF4E92DFF2716
:102F8000EE0FFF1FE55DF74F8591949128173907E4
:102F900020F49394F3E6F91588F76BE201C060E240
:102FA00081E00E94E112892D0E9419179FE0A92E4D
:102FB000A82220E3A20E182F12951F70120F60E2B4
:102FC00080E00E94E112612F82E00E94E1126A2DEE
:102FD00083E00E94E1126AE284E00E94E11263E46D
:102FE00040C1843009F044C1E92DFF27EE0FFF1FD7
:102FF000ED53F74F859194918217930720F09394A6
:103000008DE8891588F7892D0E942B17EC0193E62E
:10301000991560F46BE280E00E94E1128D2F9927F0
:1030200087FD9A95182F105D612F05C060E280E042
:103030000E94E1126BE281E00E94E1121FE0A12EEA
:10304000AC22E0E3AE0EB4E0D595C795BA95E1F7B2
:103050008C2F8F708E0F682F82E00E94E1126A2DF4
:1030600083E00E94E1126AE284E00E94E11266E4D9
:10307000F8C080917C00813009F0BEC0E90182E097
:103080000E944A170E9452179C01E92DFF27EE0F5C
:10309000FF1FE352F64F859194918217930720F416
:1030A0009394F6E1F91588F7992029F486EF98E2D0
:1030B000A4E3B0E419C025E1291528F48AEB99E4CA
:1030C000ACE3B0E411C0292D3327220F331F220FA8
:1030D000331F295F354FF901E590F490F9013296DD
:1030E00005911491D801C70180935E0190935F010F
:1030F000A0936001B0936101F1E09F2E90927C005B
:10310000CE01AA2797FDA095BA2FBC01CD010E9440
:10311000211A7B018C0180915E0190915F01A09149
:103120006001B09161019C01AD01C801B7010E942D
:103130006A1ADC01CB0120E030E040E85AE3BC0130
:10314000CD010E946A1ADC01CB0120E030E040ECA6
:1031500050E4BC01CD010E946A1A7B018C010E94DF
:10316000041A5B016C01862F9927AA2797FDA09569
:10317000BA2FBC01CD010E94211ADC01CB019C01B8
:10318000AD01C801B7010E94C119DC01CB0120E0EB
:1031900030E048EC52E4BC01CD010E946A1ADC0127
:1031A000CB01BC01CD010E94041A7B018C018A2D48
:1031B0000E941917A82EFFE0AF2220E3A20E8E2D49
:1031C0000E941917182F12951F70105D60E280E0A1
:1031D0000E94E11260E2892D0E94E11260E282E029
:1031E0000E94E1126A2D83E00E94E11266E584E00C
:1031F0000E94E112612F35C0C0917C00C230C1F540
:10320000809179000E94191780917800982F9F7003
:10321000E0E3AE2EA90EE9E3EA1518F477E3A72E52
:10322000A90E682F62956F70162F105D1A3308F083
:10323000195F61E4892D0E94E11264E481E00E943B
:10324000E11263E48C2F0E94E11280917900805D8D
:10325000682F83E00E94E112612F84E00E94E11256
:103260006A2D85E00E94E11260E086E00E94E11292
:10327000DF91CF911F910F91FF90EF90DF90CF9052
:10328000BF90AF909F900895CF93C82F6091630136
:10329000662351F01092630180E00E944A178AE889
:1032A00097E10E943F0A03C081E00E94F612C330FA
:1032B00051F48AE897E10E945E0A81E080936301FD
:1032C0008CE390E016C0C43039F480916201843000
:1032D00049F0C09362010BC0C53049F4809162018E
:1032E000843011F483E001C084E0809362018DE3B7
:1032F00090E0CF910895CF93C82F60916401662329
:1033000051F01092640181E00E944A178AE897E127
:103310000E943F0A03C081E00E94F612C33051F4BC
:103320008AE897E10E945E0A81E08093640186E466
:1033300090E002C087E490E0CF910895CF93C82F2A
:1033400060916501662351F01092650182E00E9450
:103350004A178AE897E10E943F0A03C081E00E9471
:10336000F612C33051F48AE897E10E945E0A81E0C8
:103370008093650180E590E002C081E590E0CF9107
:1033800008955058192E84D001D06AC0BA17620728
:10339000730784079507B1F188F40EF410940B2E8F
:1033A000BA2FA02D062E622F202D072E732F302D21
:1033B000082E842F402D092E952F502DFF275523A1
:1033C000B9F0591B49F0573E98F046953795279527
:1033D000A795F0405395C9F776F0BA0F621F731F97
:1033E000841F30F4879577956795B795F04093954E
:1033F00017FA0F2E0895BF1BBB27BA0B620B730B76
:10340000840BF6CFDEF660C097FB4ED09F3738F0C6
:10341000FEE9F91B982F872F762F6B2F05C051C01F
:103420009695879577956795F150D0F73EF49095EE
:103430008095709561957F4F8F4F9F4F0895E894C9
:1034400003C097FB0EF4F3DFB62F672F782F892F79
:103450009EE9002405C09A95BB0F661F771F881F41
:1034600011249923A1F08823B2F79F3F59F0BB0F95
:1034700048F421F4002011F460FF04C06F5F7F4F17
:103480008F4F9F4F881F9795879597F9089519C07B
:10349000052E092607FA440F551F5F3F79F0AA272A
:1034A000A51708F051E04795880F991F9F3F31F00D
:1034B000BB27B91708F091E0879508959F919F91D8
:1034C00057C066277727882799270895592F482FAF
:1034D000372F262FDDDF01D0C3CF992339F05523B5
:1034E00029F09F575F57950F13F4CAF1EDCF91580C
:1034F0009F3FE1F3A62F00241124BB276627552701
:10350000F8E0A69520F4020E131EB41F651F220FCB
:10351000331F441F551FFA95A1F7F8E0E72F7727CF
:10352000F8E0E69520F4130EB41F651F7A1F330FE1
:10353000441F551FAA1FFA95A1F7F82F8827F69563
:1035400020F4B40F651F7A1F8E1F440F551FAA1F4A
:10355000EE1FFF23A1F788231AF4939539F408C0CE
:10356000000C111CBB1F661F771F881F01280895C0
:103570009FEF80EC0895AA1BBB1B51E107C0AA1F57
:10358000BB1FA617B70710F0A61BB70B881F991F04
:0E3590005A95A9F780959095BC01CD0108953C
:10359E001E0101010101010101D503880446056CDC
:1035AE000682060000CB037B043E0564067A060005
:1035BE0000500101001F1C1F1E1F1E1F1F1E1F1E5D
:1035CE001F0C0102030405060708090A0B0C010271
:1035DE00030405060708090A0B0168076F0776073B
:1035EE007D078307890701010102010F01039A99E3
:0635FE0039400301010148
:00000001FF
